:200000000C9461000C947E000C947E000C947E000C947E000C947E000C947E000C947E000D
:200020000C947E000C947E000C947E000C947E000C947E000C947E000C947E000C947E00D0
:200040000C947D010C947E000C947E000C947E000C947E000C947E000C947E000C947E00B0
:200060000C947E000C947E0000000000240027002A0000000000250028002B000000000057
:20008000230026002900040404040404040402020202020203030303030301020408102071
:2000A0004080010204081020010204081020000000070002010000030406000000000000EB
:2000C000000011241FBECFEFD4E0DEBFCDBF11E0A0E0B1E0EEE6F6E002C005900D92A230FF
:2000E000B107D9F711E0A2E0B1E001C01D92AE30B107E1F70E940F030C9435030C9400006A
:200100000F931F93CF93DF9381E10E94C20210E0009709F011E082E10E94C202009709F025
:200120001260809100011817D9F0112361F0113029F0123041F0133089F408C010930301C2
:20014000109304010BC01092040108C081E080930401809303018FE1809302011093000103
:20016000113061F0123031F1133061F1809104018F5F80930401C4EFD1E061C0909103012E
:2001800080910401992341F0803121F41092030188E00BC0880F09C0813021F410930301F0
:2001A00082E003C090E09595879580930401C8ECD0E045C080910401809580930401CAEFE7
:2001C000D0E03DC090910301809104019923B9F0282F30E084FF0FC0803131F488E18093C7
:2001E00004011092030115C090910201990F9093020189231AC0220F331F21601CC0282FD0
:2002000030E080FF15C0813041F410930401809303018FE18093020110C02091020130E0BB
:20022000359527952093020182238093040105C035952795206120930401C0E9D1E0009156
:20024000040110E0B8016170707086E00E946F02B80176956795617087E00E946F02B80102
:200260007695679576956795617088E00E946F02B80193E0769567959A95E1F7617089E0B0
:200280000E946F02B80184E0769567958A95E1F761708AE00E946F02BE01882777FD8095EB
:2002A000982F0E94E801DF91CF911F910F91089586E061E00E944A0287E061E00E944A0204
:2002C00088E061E00E944A0289E061E00E944A028AE061E00E944A0281E160E00E944A02C6
:2002E00081E161E00E946F0282E160E00E944A0282E161E00E946F0208951F920F920FB64C
:200300000F9211242F933F938F939F93AF93BF938091090190910A01A0910B01B0910C01B9
:2003200030910D010196A11DB11D232F215B2D3720F02D570196A11DB11D20930D0180930E
:20034000090190930A01A0930B01B0930C018091050190910601A0910701B091080101967D
:20036000A11DB11D8093050190930601A0930701B0930801BF91AF919F918F913F912F91B7
:200380000F900FBE0F901F9018953FB7F8946091050170910601809107019091080126B557
:2003A000A89B06C02F3F21F06F5F7F4F8F4F9F4F3FBF982F872F762F6627620F711D811D03
:2003C000911D26E030E040E050E00E9416030895EF92FF920F931F93CF93DF937B018C016E
:2003E0000E94C501EB010FC00E94C5016C1B7D0B83E0683E7807C0F30894E108F1080109A0
:200400001109C851DC4FE114F1040105110561F7DF91CF911F910F91FF90EF900895789449
:2004200084B5826084BD84B5816084BD85B5826085BD85B5816085BDEEE6F0E080818160C4
:200440008083E1E8F0E01082808182608083808181608083E0E8F0E0808181608083E1EB5A
:20046000F0E0808184608083E0EBF0E0808181608083EAE7F0E080818460808380818260D8
:2004800080838081816080838081806880831092C1000895282F30E0C90186569F4FFC0190
:2004A0009491F901EA57FF4FE491EE23B9F0F0E0EE0FFF1FE859FF4FA591B491662341F4AC
:2004C0002FB7F8948C91909589238C932FBF08952FB7F8948C91892B8C932FBF0895482FAE
:2004E00050E0CA0182559F4FFC0194919A0126563F4FF9012491FA01EA57FF4FE491EE23B6
:2005000009F43FC0992331F1933021F4909180009F7705C0943031F4909180009F7D9093E4
:20052000800018C0913019F494B59F7704C0923021F494B59F7D94BD0DC0963021F490911C
:20054000B0009F7705C0973029F49091B0009F7D9093B000F0E0EE0FFF1FEE58FF4FA591B7
:20056000B491662341F49FB7F8948C91209582238C939FBF08959FB7F8948C91822B8C933A
:200580009FBF0895282F30E0C90182559F4FFC019491A90146565F4FFA014491F901EA5749
:2005A000FF4FE491EE2319F420E030E036C0992331F1933021F4909180009F7705C094305E
:2005C00031F4909180009F7D9093800018C0913019F494B59F7704C0923021F494B59F7D91
:2005E00094BD0DC0963021F49091B0009F7705C0973029F49091B0009F7D9093B000F0E0E2
:20060000EE0FFF1FE458FF4FA591B4918C9120E030E0842311F021E030E0C90108950E94CB
:200620000F020E9458010E948000FDCF629FD001739FF001829FE00DF11D649FE00DF11DD1
:20064000929FF00D839FF00D749FF00D659FF00D9927729FB00DE11DF91F639FB00DE11DDB
:20066000F91FBD01CF0111240895F894FFCF0400FFFFFFFFFFFFFFFFFFFFFFFFFFFFFFFFB4
:2006800050E00E941A0504C0E885F98510829401EC81FD813083EE81FF812083EA85FB8574
:2006A000808121E030E0A9010E8402C0440F551F0A94E2F7842B8083EA85FB858081A901A0
:2006C0000F8402C0440F551F0A94E2F7842B8083EA85FB858081088802C0220F331F0A9472
:2006E000E2F7822B8083DF91CF911F910F91FF90EF90DF90BF90AF909F908F900895FC015E
:2007000022813381F901E058FF4F8081918180589F4F2E573F4FF90120813181821B930B8E
:2007200060E870E00E94E5040895FC0182819381FC01EE57FF4F20813181FC01E058FF4F7F
:20074000408151814217530719F42FEF3FEF05C0820F931FFC01208130E0C9010895DC0100
:2007600012962D913C911397F901EE57FF4F80819181D901A058BF4F4D915C91119748174A
:20078000590719F42FEF3FEF0CC0280F391FD9012C91019660E870E00E94E50491838083DD
:2007A00030E0C9010895DC0112968D919C911397FC01E058FF4F8E579F4FDC018D919C91CA
:2007C0001197918380830895FC01A085B18521898C9190E0022E02C0959587950A94E2F77F
:2007E00080FFF6CF0484F585E02D6083089584E091E0909397018093960182E191E09093F5
:2008000099018093980185EC90E090939B0180939A0184EC90E090939D0180939C0180EC87
:2008200090E090939F0180939E0181EC90E09093A1018093A00186EC90E09093A3018093C1
:20084000A20184E08093A40183E08093A50187E08093A60185E08093A70181E08093A8015F
:2008600008951F920F920FB60F921124EF92FF920F931F932F933F934F935F938F939F93CC
:20088000AF93BF93E090AD01F090AE010091AF011091B0019091B101A80197012E5F3F4FB5
:2008A0004F4F5F4F892F8A5F8D3738F08D57A80197012D5F3F4F4F4F5F4F8093B10120935C
:2008C000AD013093AE014093AF015093B0018091A9019091AA01A091AB01B091AC010196F8
:2008E000A11DB11D8093A9019093AA01A093AB01B093AC01BF91AF919F918F915F914F9162
:200900003F912F911F910F91FF90EF900F900FBE0F901F901895789484B5826084BD84B5E1
:20092000816084BD85B5826085BD85B5816085BDEEE6F0E0808181608083E1E8F0E0108226
:20094000808182608083808181608083E0E8F0E0808181608083E1EBF0E0808184608083CB
:20096000E0EBF0E0808181608083EAE7F0E0808184608083808182608083808181608083A3
:200980008081806880831092C1000895629FD001739FF001829FE00DF11D649FE00DF11D7C
:2009A000929FF00D839FF00D749FF00D659FF00D9927729FB00DE11DF91F639FB00DE11D78
:2009C000F91FBD01CF011124089597FB092E07260AD077FD04D049D006D000201AF4709565
:2009E00061957F4F0895F6F7909581959F4F0895A1E21A2EAA1BBB1BFD010DC0AA1FBB1F0F
:200A0000EE1FFF1FA217B307E407F50720F0A21BB30BE40BF50B661F771F881F991F1A94AF
:200A200069F760957095809590959B01AC01BD01CF01089597FB092E05260ED057FD04D0B4
:200A4000D7DF0AD0001C38F450954095309521953F4F4F4F5F4F0895F6F7909580957095E6
:200A600061957F4F8F4F9F4F0895AA1BBB1B51E107C0AA1FBB1FA617B70710F0A61BB70B14
:200A8000881F991F5A95A9F780959095BC01CD010895EE0FFF1F0590F491E02D0994F8949B
:200AA000FFCF00000000E4031D0136017F03AF03D3039503FFFFFFFFFFFFFFFFFFFFFFFF96
:200AC000FFFFFFFFFFFFFFFFFFFFFFFFFFFFFFFFFFFFFFFFFFFFFFFFFFFFFFFFFFFFFFFF36
:200AE000FFFFFFFFFFFFFFFFFFFFFFFFFFFFFFFFFFFFFFFFFFFFFFFFFFFFFFFFFFFFFFFF16
:200B0000FFFFFFFFFFFFFFFFFFFFFFFFFFFFFFFFFFFFFFFFFFFFFFFFFFFFFFFFFFFFFFFFF5
:200B2000FFFFFFFFFFFFFFFFFFFFFFFFFFFFFFFFFFFFFFFFFFFFFFFFFFFFFFFFFFFFFFFFD5
:203800000C94341C0C94511C0C94511C0C94511C0C94511C0C94511C0C94511C0C94511C5D
:203820000C94511C0C94511C0C94511C0C94511C0C94511C0C94511C0C94511C0C94511C20
:203840000C94511C0C94511C0C94511C0C94511C0C94511C0C94511C0C94511C0C94511C00
:203860000C94511C0C94511C11241FBECFEFD4E0DEBFCDBF11E0A0E0B1E0E2E3FFE302C016
:2038800005900D92A230B107D9F712E0A2E0B1E001C01D92AD30B107E1F70E94271D0C9432
:2038A000971F0C94001C282F2595259525952595205D8F708A3074F0895A9091C00095FF65
:2038C000FCCF2093C6009091C00095FFFCCF8093C6000895805DF1CF9091C00095FFFCCF11
:2038E0008093C6000895EF92FF920F931F93EE24FF2487018091C00087FD17C00894E11C6A
:20390000F11C011D111D89E6E81689E8F80689E0080780E0180770F3E0910401F09105011B
:2039200009958091C00087FFE9CF8091C6001F910F91FF90EF9008950E94731C9091C000F6
:2039400095FFFCCF8093C600813624F480330CF080530895875508951F930E949C1C182F75
:203960000E949C1C1295107F810F1F9108951F93182F882321F00E94731C1150E1F71F910B
:2039800008951F93182F0E94731C803249F0809103018F5F809303018530C1F01F910895A8
:2039A0008091C00085FFFCCF84E18093C6008091C00085FFFCCF1093C6008091C00085FFCB
:2039C000FCCF80E18093C6001F910895E0910401F091050109951F9108950E94731C8032CA
:2039E00041F0809103018F5F80930301853081F008958091C00085FFFCCF84E18093C6005B
:203A00008091C00085FFFCCF80E18093C6000895E0910401F0910501099508954AEF50E00E
:203A20008823A1F02A9A28EE33E0FA013197F1F721503040D1F72A9828EE33E0FA0131975B
:203A4000F1F721503040D1F7815061F70895EF92FF920F931F93CF93DF9394B714BE8091A7
:203A600060008861809360001092600091FF59C28FE18093C4001092C50088E18093C100F2
:203A800086E08093C2005098589A229A81E00E940E1D64E1E62E50E1F52E0E94731C803396
:203AA000B1F18133B9F1803409F476C0813409F47BC0823449F1853409F488C0803539F165
:203AC000823529F1813509F494C1853509F490C0863509F481C0843609F40FC1843709F4CE
:203AE000B7C0853709F48FC0863709F46BC0809103018F5F80930301853079F6E0910401AE
:203B0000F09105010995C9CF84E10E94B71C0E94ED1CC3CF0E94731C803249F78091C000DD
:203B200085FFFCCFE092C6008091C00085FFFCCF81E48093C6008091C00085FFFCCF86E515
:203B40008093C6008091C00085FFFCCF82E58093C6008091C00085FFFCCF80E28093C600D1
:203B60008091C00085FFFCCF89E48093C6008091C00085FFFCCF83E58093C6008091C000AD
:203B800085FFFCCF80E58093C6008091C00085FFFCCFF092C60081CF0E94731C863808F4F5
:203BA000B6CF0E94731CB3CF0E94731C803809F441C1813809F43AC1823809F433C18839C8
:203BC00009F42CC180E00E94C11C67CF85E00E94B71C0E94ED1C61CF0E94731C803309F450
:203BE0000EC183E00E94B71C80E00E94C11C55CF0E94731C809306010E94731C8093070184
:203C00000E94ED1C4ACF0E94731C803209F06FCF8091C00085FFFCCFE092C6008091C0009D
:203C200085FFFCCF8EE18093C6008091C00085FFFCCF84E98093C6008091C00085FFFCCF67
:203C400086E08093C6008091C00085FFFCCFA1CF0E94731C809309020E94731C80930802F8
:203C60008091060190910701880F991F90930701809306010E94731C853409F4A9C080910E
:203C80000C028E7F80930C020E94731C803209F004CF8091C00085FFFCCFE092C600209130
:203CA00008023091090280910C02782F7170682F62704091060150910701FA0180E090E092
:203CC0008217930708F08AC0772361F4662339F4A491B091C000B5FFFCCFA093C600019685
:203CE0003196EECFF999FECFF2BDE1BDF89AA0B5B091C000B5FFFCCFF0CF0E94731C80932A
:203D000009020E94731C8093080280910C028E7F80930C020E94731C853429F480910C02D7
:203D2000816080930C028091080290910902009789F000E010E00E94731CF801E85FFE4F9C
:203D400080830F5F1F4F80910802909109020817190788F30E94731C803209F0C8CE809100
:203D60000C02817009F472C02091060130910701220F331F30930701209306016091080291
:203D80007091090261157105C1F0E8E0F1E0DB01AE0FBF1FC901F999FECF92BD81BD4191E2
:203DA00040BDFA9AF99A0196EA17FB07A1F7260F371F30930701209306018091C00085FF48
:203DC000FCCFE092C6008091C00085FFFCCFE1CE80910C02816080930C0256CF240F351F44
:203DE00030930701209306018091C00085FFFCCFD0CE0E94ED1C88E080936000FFCF0E948A
:203E0000731C0E94731C082F0E94731C0023D1F00130A1F086E00E94C11C3FCE83E00E94DD
:203E2000C11C3BCE80E10E94C11C37CE81E00E94C11C33CE82E00E94C11C2FCE84E90E94E9
:203E4000C11C2BCE8EE10E94C11C27CE80910701880F880B817080930B028091060190911C
:203E60000701880F991F90930701809306018091080280FF09C08091080290910902019665
:203E80009093090280930802F894F999FECF1127E0910601F0910701C8E0D1E0809108023F
:203EA00090910902103091F40091570001700130D9F303E000935700E89500915700017018
:203EC0000130D9F301E100935700E895099019900091570001700130D9F301E00093570039
:203EE000E8951395103498F011270091570001700130D9F305E000935700E895009157000F
:203F000001700130D9F301E100935700E8953296029709F0C7CF103011F00296E5CF112438
:143F20004CCFE0910401F09105010995A1CDF894FFCF80008F
:00000001FF
